 sgx_clipblit_test

 Timestamp is 4be8c2d4 (Tue May 11 11:37:08 2010)

 Preferred load address is 00010000

 Start         Length     Name                   Class
 0001:00000000 00000004H .CRT$XCA                CODE
 0001:00000004 00000004H .CRT$XCZ                CODE
 0001:00000008 00000004H .CRT$XIA                CODE
 0001:0000000c 00000004H .CRT$XIZ                CODE
 0001:00000010 00000004H .CRT$XPA                CODE
 0001:00000014 00000004H .CRT$XPZ                CODE
 0001:00000018 00000004H .CRT$XTA                CODE
 0001:0000001c 00000004H .CRT$XTZ                CODE
 0001:00000020 00000c1fH .rdata                  CODE
 0001:00000c40 0000002eH .rdata$debug            CODE
 0001:00000c70 00001708H .text                   CODE
 0001:00002378 0000001cH .xdata                  CODE
 0001:00002394 00000028H .idata$2                CODE
 0001:000023bc 00000014H .idata$3                CODE
 0001:000023d0 000000b4H .idata$4                CODE
 0001:00002484 0000013aH .idata$6                CODE
 0001:000025be 00000000H .edata                  CODE
 0002:00000000 000000b4H .idata$5                DATA
 0002:000000b8 000984ccH .data                   DATA
 0002:00098584 00000010H .bss                    DATA
 0003:00000000 000000b0H .pdata                  DATA

  Address         Publics by Value              Rva+Base       Lib:Object

 0000:00000000       ___safe_se_handler_table   00000000     <absolute>
 0000:00000000       ___safe_se_handler_count   00000000     <absolute>
 0001:00000000       __xc_a                     00011000     corelib0:crt0init.obj
 0001:00000004       __xc_z                     00011004     corelib0:crt0init.obj
 0001:00000008       __xi_a                     00011008     corelib0:crt0init.obj
 0001:0000000c       __xi_z                     0001100c     corelib0:crt0init.obj
 0001:00000010       __xp_a                     00011010     corelib0:crt0init.obj
 0001:00000014       __xp_z                     00011014     corelib0:crt0init.obj
 0001:00000018       __xt_a                     00011018     corelib0:crt0init.obj
 0001:0000001c       __xt_z                     0001101c     corelib0:crt0init.obj
 0001:0000003c       ??_C@_0DH@LFOMPFHH@?9?9?9?9?9?9?9?9?9?9?9?9?9?9?9?9?9?5SGX?5ClipBlit?5t@ 0001103c     sgx_clipblit_test.obj
 0001:00000074       ??_C@_0DH@IDEKHJEN@?9?9?9?9?9?9?9?9?9?9?9?9?9?9?9?9?9?9?9?9?9?9?9?9?5End?5?9?9?9@ 00011074     sgx_clipblit_test.obj
 0001:000000ac       ??_C@_0BP@GJLKNMBD@Destroy?5the?5transfer?5context?3?6?$AA@ 000110ac     sgx_clipblit_test.obj
 0001:000000cc       ??_C@_0DD@GODBIEMM@Display?5Class?5API?3?5unmap?5display@ 000110cc     sgx_clipblit_test.obj
 0001:00000100       ??_C@_0DJ@OPOMFNMC@Polling?5for?5destination?5surface?5@ 00011100     sgx_clipblit_test.obj
 0001:0000013c       ??_C@_0CN@CJJNALAI@Attempt?5to?5create?5transfer?5conte@ 0001113c     sgx_clipblit_test.obj
 0001:0000016c       ??_C@_04LNELOFCG@?5OK?6?$AA@ 0001116c     sgx_clipblit_test.obj
 0001:00000174       ??_C@_0CP@IFAFGPME@Display?5Class?5API?3?5map?5display?5s@ 00011174     sgx_clipblit_test.obj
 0001:000001a4       ??_C@_0M@FBGHFOFL@?5FAIL?5?9?5?$CFs?6?$AA@ 000111a4     sgx_clipblit_test.obj
 0001:000001b0       ??_C@_0DH@GJHJBGDL@?9?9?9?9?9?9?9?9?9?9?9?9?9?9?9?9?9?5SGX?5CLipBlit?5t@ 000111b0     sgx_clipblit_test.obj
 0001:000001e8       ??_C@_0DH@FEMFBJEL@?9?9?9?9?9?9?9?9?9?9?9?9?9?9?9?9?9?9?9?9?9?9?5Start?5?9?9?9@ 000111e8     sgx_clipblit_test.obj
 0001:00000220       ??_C@_0DE@BODOPOHG@Display?5Class?5API?3?5get?5the?5syste@ 00011220     sgx_clipblit_test.obj
 0001:00000258       ??_C@_1KE@BDGMONOJ@?$AAH?$AA?3?$AA?2?$AAW?$AAI?$AAN?$AAC?$AAE?$AA6?$AA0?$AA0?$AA?2?$AAP?$AAL?$AAA?$AAT?$AAF?$AAO?$AAR?$AAM?$AA?2?$AAS?$AAM?$AAD?$AAK?$AAV?$AA2?$AA1?$AA0?$AA?2?$AAS?$AAR@ 00011258     wince_unittests.obj
 0001:000002fc       ??_C@_1CI@OHCJFJPM@?$AAE?$AAR?$AAR?$AAO?$AAR?$AA?3?$AA?5?$AA?$CF?$AAs?$AA?5?$AAl?$AAi?$AAn?$AAe?$AA?5?$AA?$CF?$AAd?$AA?3?$AA?5?$AA?$AA@ 000112fc     wince_unittests.obj
 0001:00000324       ??_C@_1CK@MPGKAOE@?$AA?$CI?$AAe?$AAr?$AAr?$AAo?$AAr?$AA?5?$AAc?$AAo?$AAd?$AAe?$AA?3?$AA?5?$AA?$CF?$AAd?$AA?$CJ?$AA?3?$AA?5?$AA?$CF?$AAs?$AA?$AA@ 00011324     wince_unittests.obj
 0001:00000350       ??_C@_1M@DMCDIEDK@?$AAP?$AAK?$AAM?$AA1?$AA?3?$AA?$AA@ 00011350     wince_unittests.obj
 0001:0000035c       ??_C@_0L@GPAGIAIC@?9disablepm?$AA@ 0001135c     wince_unittests.obj
 0001:00000368       ??_C@_07FBLHGNAH@app?4exe?$AA@ 00011368     wince_unittests.obj
 0001:00000370       ??_C@_0BD@FOHFKAOE@INVALID?5ERROR?5CODE?$AA@ 00011370     sgx_unittest_utils.obj
 0001:00000384       ??_C@_09KMCHPOPM@PVRSRV_OK?$AA@ 00011384     sgx_unittest_utils.obj
 0001:00000390       ??_C@_0BF@KHEAJDEG@PVRSRV_ERROR_GENERIC?$AA@ 00011390     sgx_unittest_utils.obj
 0001:000003a8       ??_C@_0BL@BOENCAIM@PVRSRV_ERROR_OUT_OF_MEMORY?$AA@ 000113a8     sgx_unittest_utils.obj
 0001:000003c4       ??_C@_0BN@IHBDMIPO@PVRSRV_ERROR_TOO_FEW_BUFFERS?$AA@ 000113c4     sgx_unittest_utils.obj
 0001:000003e4       ??_C@_0BO@EGNEIFEA@PVRSRV_ERROR_SYMBOL_NOT_FOUND?$AA@ 000113e4     sgx_unittest_utils.obj
 0001:00000404       ??_C@_0BL@BKMGFOLH@PVRSRV_ERROR_OUT_OF_HSPACE?$AA@ 00011404     sgx_unittest_utils.obj
 0001:00000420       ??_C@_0BM@LGNAOM@PVRSRV_ERROR_INVALID_PARAMS?$AA@ 00011420     sgx_unittest_utils.obj
 0001:0000043c       ??_C@_0BN@MGJEIKFE@PVRSRV_ERROR_TILE_MAP_FAILED?$AA@ 0001143c     sgx_unittest_utils.obj
 0001:0000045c       ??_C@_0BK@JHPIKHJG@PVRSRV_ERROR_INIT_FAILURE?$AA@ 0001145c     sgx_unittest_utils.obj
 0001:00000478       ??_C@_0CE@POPMCOCG@PVRSRV_ERROR_CANT_REGISTER_CALLB@ 00011478     sgx_unittest_utils.obj
 0001:0000049c       ??_C@_0BM@COIEDMNF@PVRSRV_ERROR_INVALID_DEVICE?$AA@ 0001149c     sgx_unittest_utils.obj
 0001:000004b8       ??_C@_0BH@OEOFFCIM@PVRSRV_ERROR_NOT_OWNER?$AA@ 000114b8     sgx_unittest_utils.obj
 0001:000004d0       ??_C@_0BJ@PHFCJIBD@PVRSRV_ERROR_BAD_MAPPING?$AA@ 000114d0     sgx_unittest_utils.obj
 0001:000004ec       ??_C@_0BF@KGIMOMJE@PVRSRV_ERROR_TIMEOUT?$AA@ 000114ec     sgx_unittest_utils.obj
 0001:00000504       ??_C@_0BI@CDPBDDFH@PVRSRV_ERROR_NO_PRIMARY?$AA@ 00011504     sgx_unittest_utils.obj
 0001:0000051c       ??_C@_0BP@FMELGOJO@PVRSRV_ERROR_FLIP_CHAIN_EXISTS?$AA@ 0001151c     sgx_unittest_utils.obj
 0001:0000053c       ??_C@_0BN@JMHJCLJP@ERROR_CANNOT_ACQUIRE_SYSDATA?$AA@ 0001153c     sgx_unittest_utils.obj
 0001:0000055c       ??_C@_0BL@JPEIBKNH@PVRSRV_ERROR_SCENE_INVALID?$AA@ 0001155c     sgx_unittest_utils.obj
 0001:00000578       ??_C@_0BK@JAAFMMBM@PVRSRV_ERROR_STREAM_ERROR?$AA@ 00011578     sgx_unittest_utils.obj
 0001:00000594       ??_C@_0BP@LELIGCIL@PVRSRV_ERROR_INVALID_INTERRUPT?$AA@ 00011594     sgx_unittest_utils.obj
 0001:000005b4       ??_C@_0CB@HFGDLHLE@PVRSRV_ERROR_FAILED_DEPENDENCIES@ 000115b4     sgx_unittest_utils.obj
 0001:000005d8       ??_C@_0BP@PFBLKCEO@PVRSRV_ERROR_CMD_NOT_PROCESSED?$AA@ 000115d8     sgx_unittest_utils.obj
 0001:000005f8       ??_C@_0BJ@PHLIKBPN@PVRSRV_ERROR_CMD_TOO_BIG?$AA@ 000115f8     sgx_unittest_utils.obj
 0001:00000614       ??_C@_0CE@FHHHLEGE@PVRSRV_ERROR_DEVICE_REGISTER_FAI@ 00011614     sgx_unittest_utils.obj
 0001:00000638       ??_C@_0BI@JBKNPCOM@PVRSRV_ERROR_FIFO_SPACE?$AA@ 00011638     sgx_unittest_utils.obj
 0001:00000650       ??_C@_0BJ@IIGHNIEG@PVRSRV_ERROR_TA_RECOVERY?$AA@ 00011650     sgx_unittest_utils.obj
 0001:0000066c       ??_C@_0BN@BKNBJNB@PVRSRV_ERROR_INDOSORLOWPOWER?$AA@ 0001166c     sgx_unittest_utils.obj
 0001:0000068c       ??_C@_0BM@MCHBLHIP@PVRSRV_ERROR_TOOMANYBUFFERS?$AA@ 0001168c     sgx_unittest_utils.obj
 0001:000006a8       ??_C@_0BL@FINKNLDE@PVRSRV_ERROR_NOT_SUPPORTED?$AA@ 000116a8     sgx_unittest_utils.obj
 0001:000006c4       ??_C@_0CA@KIDKOOGL@PVRSRV_ERROR_PROCESSING_BLOCKED?$AA@ 000116c4     sgx_unittest_utils.obj
 0001:000006e4       ??_C@_0BG@OJDNODAO@PVRSRV_ERROR_NO_MUTEX?$AA@ 000116e4     sgx_unittest_utils.obj
 0001:000006fc       ??_C@_0CA@NBGAMPKE@PVRSRV_ERROR_CANNOT_FLUSH_QUEUE?$AA@ 000116fc     sgx_unittest_utils.obj
 0001:0000071c       ??_C@_0CE@NLLBGAEA@PVRSRV_ERROR_CANNOT_GET_QUEUE_SP@ 0001171c     sgx_unittest_utils.obj
 0001:00000740       ??_C@_0CG@FCILKACH@PVRSRV_ERROR_CANNOT_GET_RENDERDE@ 00011740     sgx_unittest_utils.obj
 0001:00000768       ??_C@_0BD@COEEPPOL@PVRSRV_ERROR_RETRY?$AA@ 00011768     sgx_unittest_utils.obj
 0001:0000077c       ??_C@_0BB@EIDKNEMM@?5FAIL?5?9?5?$CFs?$CI?$CFlu?$CJ?6?$AA@ 0001177c     sgx_unittest_utils.obj
 0001:00000790       ??_C@_0BJ@IMBALOKG@PVRSRV_DEVICE_ID_UNKNOWN?$AA@ 00011790     sgx_unittest_utils.obj
 0001:000007ac       ??_C@_0BH@OGEGGGCD@PVRSRV_DEVICE_ID_MSVDX?$AA@ 000117ac     sgx_unittest_utils.obj
 0001:000007c4       ??_C@_0BF@BBCLGMON@PVRSRV_DEVICE_ID_SGX?$AA@ 000117c4     sgx_unittest_utils.obj
 0001:000007dc       ??_C@_0CD@BDGFMHBG@PVRSRV_DEVICE_TYPE_EXT?5?$CI3rd?5Part@ 000117dc     sgx_unittest_utils.obj
 0001:00000800       ??_C@_0BE@GEDKFGMC@Not?5recognised?50x?$CFx?$AA@ 00011800     sgx_unittest_utils.obj
 0001:00000814       ??_C@_0BI@ICLDLMDM@?4?4?4?4?5ui32ProcessID?3?$CFlu?6?$AA@ 00011814     sgx_unittest_utils.obj
 0001:00000830       ??_C@_0EK@BPNJOJAB@?4?4?4?4?5Shared?5heap?5?$CFlu?5?9?5HeapID?30x@ 00011830     sgx_unittest_utils.obj
 0001:0000087c       ??_C@_0CL@DNLHEBLI@Attempt?5to?5create?5memory?5context@ 0001187c     sgx_unittest_utils.obj
 0001:000008a8       ??_C@_0ED@NNKEOJPF@?4?4?4?4?5Display?5dimensions?5?$CFlu?5?9?5By@ 000118a8     sgx_unittest_utils.obj
 0001:000008ec       ??_C@_0DB@DPDHNDGF@Display?5Class?5API?3?5enumerate?5dis@ 000118ec     sgx_unittest_utils.obj
 0001:00000920       ??_C@_0CK@PAKBMFJN@?4?4?4?4?5Display?5format?5?$CFlu?5?9?5Pixelf@ 00011920     sgx_unittest_utils.obj
 0001:0000094c       ??_C@_0CF@FMDFFMKC@Display?5Class?5API?3?5Get?5display?5i@ 0001194c     sgx_unittest_utils.obj
 0001:00000974       ??_C@_0O@GDPIEJBG@?4?4?4?4?5Name?3?$CFs?6?$AA@ 00011974     sgx_unittest_utils.obj
 0001:00000984       ??_C@_0BI@BLGHILNJ@?4?4?4?4?5MaxSwapChains?3?$CFlu?6?$AA@ 00011984     sgx_unittest_utils.obj
 0001:0000099c       ??_C@_0BO@POAFDAJE@?4?4?4?4?5MaxSwapChainBuffers?3?$CFlu?6?$AA@ 0001199c     sgx_unittest_utils.obj
 0001:000009bc       ??_C@_0BK@CPCAOBID@?4?4?4?4?5MinSwapInterval?3?$CFlu?6?$AA@ 000119bc     sgx_unittest_utils.obj
 0001:000009d8       ??_C@_0BK@DMGFAHCI@?4?4?4?4?5MaxSwapInterval?3?$CFlu?6?$AA@ 000119d8     sgx_unittest_utils.obj
 0001:000009f4       ??_C@_0CO@GIPBIACE@Display?5Class?5API?3?5enumerate?5dis@ 000119f4     sgx_unittest_utils.obj
 0001:00000a24       ??_C@_0CA@DAONOMAK@Display?5Class?5API?3?5open?5device?6?$AA@ 00011a24     sgx_unittest_utils.obj
 0001:00000a44       ??_C@_0CA@DGGJNKGO@?5Test?5Memory?5Allocation?5FAILED?6?$AA@ 00011a44     sgx_unittest_utils.obj
 0001:00000a64       ??_C@_0CG@MMBLEMBO@Display?5Class?5API?3?5enumerate?5dev@ 00011a64     sgx_unittest_utils.obj
 0001:00000a8c       ??_C@_0DM@CIPNLPOO@PVRSRVEnumerateDeviceClass?$CI?$CJ?5ret@ 00011a8c     sgx_unittest_utils.obj
 0001:00000ac8       ??_C@_0BJ@NLALCGOE@Getting?5SGX?5Client?5info?6?$AA@ 00011ac8     sgx_unittest_utils.obj
 0001:00000ae4       ??_C@_0BP@IDIGABKI@Attempt?5to?5acquire?5device?5?$CFd?3?6?$AA@ 00011ae4     sgx_unittest_utils.obj
 0001:00000b04       ??_C@_01EEMJAFIK@?6?$AA@   00011b04     sgx_unittest_utils.obj
 0001:00000b08       ??_C@_0BH@PPGIPGOP@?5?5?5?5?5?5?5?5?5?5?5?5?$CF04d?5?5?5?5?$HM?5?$AA@ 00011b08     sgx_unittest_utils.obj
 0001:00000b20       ??_C@_0CL@KFFMIBHA@Call?5PVRSRVConnect?5with?5a?5valid?5@ 00011b20     sgx_unittest_utils.obj
 0001:00000b4c       ??_C@_0DE@KAFOOJDI@Get?5number?5of?5devices?5from?5PVRSR@ 00011b4c     sgx_unittest_utils.obj
 0001:00000b80       ??_C@_0BK@GEDDINJE@?4?4?4?4?5Reported?5?$CFu?5devices?6?$AA@ 00011b80     sgx_unittest_utils.obj
 0001:00000b9c       ??_C@_0CD@INKLJIDI@?4?4?4?4?5Device?5Number?5?5?$HM?5Device?5Typ@ 00011b9c     sgx_unittest_utils.obj
 0001:00000bc0       ??_C@_0BP@HJNHLLEN@Destroy?5Device?5Memory?5Context?6?$AA@ 00011bc0     sgx_unittest_utils.obj
 0001:00000be0       ??_C@_0CF@DBFHMBAF@Display?5Class?5API?3?5close?5the?5dev@ 00011be0     sgx_unittest_utils.obj
 0001:00000c08       ??_C@_0BK@HGIBJBNI@Release?5SGX?5Client?5Info?3?6?$AA@ 00011c08     sgx_unittest_utils.obj
 0001:00000c24       ??_C@_0BL@JBOAKENO@Disconnect?5from?5services?3?6?$AA@ 00011c24     sgx_unittest_utils.obj
 0001:00000c78       main                       00011c78 f   sgx_clipblit_test.obj
 0001:0000116c       WinMain                    0001216c f   wince_unittests.obj
 0001:00001394       sgxut_GetErrorString       00012394 f   sgx_unittest_utils.obj
 0001:00001568       sgxut_null_dpf             00012568 f   sgx_unittest_utils.obj
 0001:0000157c       sgxut_fail_if_error        0001257c f   sgx_unittest_utils.obj
 0001:000015b8       sgxut_GetBytesPerPixel     000125b8 f   sgx_unittest_utils.obj
 0001:00001644       sgxut_fail_if_error_quiet  00012644 f   sgx_unittest_utils.obj
 0001:00001674       sgxut_print_dev_type       00012674 f   sgx_unittest_utils.obj
 0001:000016d4       sgxut_SGXInit              000126d4 f   sgx_unittest_utils.obj
 0001:00001cb8       sgxut_SGXDeInit            00012cb8 f   sgx_unittest_utils.obj
 0001:00001d78       ReleasePowerRequirement    00012d78 f   coredll:COREDLL.dll
 0001:00001d88       NKDbgPrintfW               00012d88 f   coredll:COREDLL.dll
 0001:00001d98       FormatMessageW             00012d98 f   coredll:COREDLL.dll
 0001:00001da8       GetLastError               00012da8 f   coredll:COREDLL.dll
 0001:00001db8       SetPowerRequirement        00012db8 f   coredll:COREDLL.dll
 0001:00001dc8       WideCharToMultiByte        00012dc8 f   coredll:COREDLL.dll
 0001:00001dd8       SGXDestroyTransferContext  00012dd8 f   srvclum:SRVCLUM.dll
 0001:00001de8       PVRSRVUnmapDeviceClassMemory 00012de8 f   srvclum:SRVCLUM.dll
 0001:00001df8       PVRSRVFreeDeviceMem        00012df8 f   srvclum:SRVCLUM.dll
 0001:00001e08       PVRSRVPollForValue         00012e08 f   srvclum:SRVCLUM.dll
 0001:00001e18       SGXQueueTransfer           00012e18 f   srvclum:SRVCLUM.dll
 0001:00001e28       PVRSRVMemSet               00012e28 f   srvclum:SRVCLUM.dll
 0001:00001e38       PVRSRVAllocDeviceMem       00012e38 f   srvclum:SRVCLUM.dll
 0001:00001e48       SGXCreateTransferContext   00012e48 f   srvclum:SRVCLUM.dll
 0001:00001e58       PVRSRVMapDeviceClassMemory 00012e58 f   srvclum:SRVCLUM.dll
 0001:00001e68       PVRSRVGetDCSystemBuffer    00012e68 f   srvclum:SRVCLUM.dll
 0001:00001e78       PVRSRVCreateDeviceMemContext 00012e78 f   srvclum:SRVCLUM.dll
 0001:00001e88       PVRSRVEnumDCDims           00012e88 f   srvclum:SRVCLUM.dll
 0001:00001e98       PVRSRVEnumDCFormats        00012e98 f   srvclum:SRVCLUM.dll
 0001:00001ea8       PVRSRVGetDCInfo            00012ea8 f   srvclum:SRVCLUM.dll
 0001:00001eb8       PVRSRVOpenDCDevice         00012eb8 f   srvclum:SRVCLUM.dll
 0001:00001ec8       PVRSRVEnumerateDeviceClass 00012ec8 f   srvclum:SRVCLUM.dll
 0001:00001ed8       SGXGetClientInfo           00012ed8 f   srvclum:SRVCLUM.dll
 0001:00001ee8       PVRSRVAcquireDeviceData    00012ee8 f   srvclum:SRVCLUM.dll
 0001:00001ef8       PVRSRVEnumerateDevices     00012ef8 f   srvclum:SRVCLUM.dll
 0001:00001f08       PVRSRVConnect              00012f08 f   srvclum:SRVCLUM.dll
 0001:00001f18       PVRSRVDisconnect           00012f18 f   srvclum:SRVCLUM.dll
 0001:00001f28       SGXReleaseClientInfo       00012f28 f   srvclum:SRVCLUM.dll
 0001:00001f38       PVRSRVCloseDCDevice        00012f38 f   srvclum:SRVCLUM.dll
 0001:00001f48       PVRSRVDestroyDeviceMemContext 00012f48 f   srvclum:SRVCLUM.dll
 0001:00001fd8       WinMainCRTStartup          00012fd8 f   corelib0:pegwmain.obj
 0001:000020d4       exit                       000130d4 f   corelib0:cexit.obj
 0001:000020ec       _exit                      000130ec f   corelib0:cexit.obj
 0001:0000212c       __GSHandlerCheckCommon     0001312c f   corelib0:gshandler.obj
 0001:00002168       __GSHandlerCheck           00013168 f   corelib0:gshandler.obj
 0001:0000218c       __security_init_cookie     0001318c f   corelib0:seccinit.obj
 0001:000021e8       __security_check_cookie    000131e8 f   corelib0:armsecgs.obj
 0001:000021fc       __gsfailure                000131fc f   corelib0:armsecgs.obj
 0001:00002240       _initterm                  00013240 f   corelib0:crt0dat.obj
 0001:00002274       _cinit                     00013274 f   corelib0:crt0dat.obj
 0001:000022a8       printf                     000132a8 f   corelib1:COREDLL.dll
 0001:000022b8       memcpy                     000132b8 f   corelib1:COREDLL.dll
 0001:000022c8       memset                     000132c8 f   corelib1:COREDLL.dll
 0001:000022d8       _stricmp                   000132d8 f   corelib1:COREDLL.dll
 0001:000022e8       _isctype                   000132e8 f   corelib1:COREDLL.dll
 0001:000022f8       malloc                     000132f8 f   corelib1:COREDLL.dll
 0001:00002308       wcslen                     00013308 f   corelib1:COREDLL.dll
 0001:00002318       free                       00013318 f   corelib1:COREDLL.dll
 0001:00002328       _XcptFilter                00013328 f   corelib1:COREDLL.dll
 0001:00002338       __C_specific_handler       00013338 f   corelib1:COREDLL.dll
 0001:00002348       __security_gen_cookie2     00013348 f   corelib1:COREDLL.dll
 0001:00002358       __report_gsfailure         00013358 f   corelib1:COREDLL.dll
 0001:00002368       TerminateProcess           00013368 f   coredll:COREDLL.dll
 0001:00002394       __IMPORT_DESCRIPTOR_COREDLL 00013394     coredll:COREDLL.dll
 0001:000023a8       __IMPORT_DESCRIPTOR_SRVCLUM 000133a8     srvclum:SRVCLUM.dll
 0001:000023bc       __NULL_IMPORT_DESCRIPTOR   000133bc     coredll:COREDLL.dll
 0002:00000000       __imp_ReleasePowerRequirement 00014000     coredll:COREDLL.dll
 0002:00000004       __imp_NKDbgPrintfW         00014004     coredll:COREDLL.dll
 0002:00000008       __imp_FormatMessageW       00014008     coredll:COREDLL.dll
 0002:0000000c       __imp_GetLastError         0001400c     coredll:COREDLL.dll
 0002:00000010       __imp_SetPowerRequirement  00014010     coredll:COREDLL.dll
 0002:00000014       __imp_WideCharToMultiByte  00014014     coredll:COREDLL.dll
 0002:00000018       __imp___report_gsfailure   00014018     corelib1:COREDLL.dll
 0002:0000001c       __imp___security_gen_cookie2 0001401c     corelib1:COREDLL.dll
 0002:00000020       __imp___C_specific_handler 00014020     corelib1:COREDLL.dll
 0002:00000024       __imp__XcptFilter          00014024     corelib1:COREDLL.dll
 0002:00000028       __imp_free                 00014028     corelib1:COREDLL.dll
 0002:0000002c       __imp_wcslen               0001402c     corelib1:COREDLL.dll
 0002:00000030       __imp_malloc               00014030     corelib1:COREDLL.dll
 0002:00000034       __imp__isctype             00014034     corelib1:COREDLL.dll
 0002:00000038       __imp__stricmp             00014038     corelib1:COREDLL.dll
 0002:0000003c       __imp_memset               0001403c     corelib1:COREDLL.dll
 0002:00000040       __imp_memcpy               00014040     corelib1:COREDLL.dll
 0002:00000044       __imp_printf               00014044     corelib1:COREDLL.dll
 0002:00000048       __imp_TerminateProcess     00014048     coredll:COREDLL.dll
 0002:0000004c       \177COREDLL_NULL_THUNK_DATA 0001404c     coredll:COREDLL.dll
 0002:00000050       __imp_PVRSRVOpenDCDevice   00014050     srvclum:SRVCLUM.dll
 0002:00000054       __imp_SGXGetClientInfo     00014054     srvclum:SRVCLUM.dll
 0002:00000058       __imp_PVRSRVAcquireDeviceData 00014058     srvclum:SRVCLUM.dll
 0002:0000005c       __imp_PVRSRVEnumerateDevices 0001405c     srvclum:SRVCLUM.dll
 0002:00000060       __imp_PVRSRVConnect        00014060     srvclum:SRVCLUM.dll
 0002:00000064       __imp_PVRSRVDisconnect     00014064     srvclum:SRVCLUM.dll
 0002:00000068       __imp_SGXReleaseClientInfo 00014068     srvclum:SRVCLUM.dll
 0002:0000006c       __imp_PVRSRVCloseDCDevice  0001406c     srvclum:SRVCLUM.dll
 0002:00000070       __imp_PVRSRVDestroyDeviceMemContext 00014070     srvclum:SRVCLUM.dll
 0002:00000074       __imp_PVRSRVGetDCInfo      00014074     srvclum:SRVCLUM.dll
 0002:00000078       __imp_PVRSRVEnumDCFormats  00014078     srvclum:SRVCLUM.dll
 0002:0000007c       __imp_PVRSRVEnumDCDims     0001407c     srvclum:SRVCLUM.dll
 0002:00000080       __imp_PVRSRVCreateDeviceMemContext 00014080     srvclum:SRVCLUM.dll
 0002:00000084       __imp_PVRSRVGetDCSystemBuffer 00014084     srvclum:SRVCLUM.dll
 0002:00000088       __imp_PVRSRVMapDeviceClassMemory 00014088     srvclum:SRVCLUM.dll
 0002:0000008c       __imp_SGXCreateTransferContext 0001408c     srvclum:SRVCLUM.dll
 0002:00000090       __imp_PVRSRVAllocDeviceMem 00014090     srvclum:SRVCLUM.dll
 0002:00000094       __imp_PVRSRVMemSet         00014094     srvclum:SRVCLUM.dll
 0002:00000098       __imp_SGXQueueTransfer     00014098     srvclum:SRVCLUM.dll
 0002:0000009c       __imp_PVRSRVPollForValue   0001409c     srvclum:SRVCLUM.dll
 0002:000000a0       __imp_PVRSRVFreeDeviceMem  000140a0     srvclum:SRVCLUM.dll
 0002:000000a4       __imp_PVRSRVUnmapDeviceClassMemory 000140a4     srvclum:SRVCLUM.dll
 0002:000000a8       __imp_SGXDestroyTransferContext 000140a8     srvclum:SRVCLUM.dll
 0002:000000ac       __imp_PVRSRVEnumerateDeviceClass 000140ac     srvclum:SRVCLUM.dll
 0002:000000b0       \177SRVCLUM_NULL_THUNK_DATA 000140b0     srvclum:SRVCLUM.dll
 0002:000000b8       londoneye160_data          000140b8     sgx_clipblit_test.obj
 0002:0009857c       __security_cookie          000ac57c     corelib0:seccinit.obj
 0002:00098580       __security_cookie_complement 000ac580     corelib0:seccinit.obj
 0002:00098584       pfnRegisteredWndProc       000ac584     wince_unittests.obj
 0002:00098588       _exitflag                  000ac588     corelib0:cexit.obj
 0002:0009858c       __onexitend                000ac58c     <common>
 0002:00098590       __onexitbegin              000ac590     <common>

 entry point at        0001:00001fd8

 Static symbols

 0001:00001f60       WinMainCRTStartupHelper    00012f60 f   corelib0:pegwmain.obj
 0001:0000200c       doexit                     0001300c f   corelib0:cexit.obj
